:020000040000FA
:02000000A8282E
:08000800A400030EA50004088A
:10001000F0000A08F1008A01831203138B1A0B1DEA
:1000200014287E200B1175280B1A8B1C1A289C2073
:100030008B1075288B190B1C20289D200B10752800
:100040000B1F752883160C1F2B2883120C1F2B28BF
:100050009E200C13752883168C1E332883128C1E49
:1000600033289F20752883160C1E3C2883120C1EF3
:100070003C28A0200C12752883168C1D452883125D
:100080008C1D4528A1208C11752883160C1D4E2827
:1000900083120C1D4E28A2200C11752883168C1C6F
:1000A000572883128C1C5728A3208C107528831680
:1000B0000C1C602883120C1C6028A4200C107528CE
:1000C00083160D1E692883120D1E6928A5200D12A6
:1000D000752883168D1D722883128D1D7228A62007
:1000E0008D1175288312A7200D1071088A007008E1
:1000F0008400250E8300A40E240E0900A00B080026
:10010000043085063330A00081309F00E530A10027
:10011000A10B88281F15000000001F198B281E083E
:10012000F039A202031D20210319CC20A2002030A7
:10013000A100A10B99280800080008000800080089
:10014000080008000800080008000800080008006F
:100150008312031385018601870183160E309F00E9
:100160003B308500003086000030870087308100FA
:1001700020308B0000308C0000308D008312203046
:1001800084008001840A841FC1283330A0008C01C0
:100190008D018B17CB28CB28A4000308A5000A08E3
:1001A000A600A30A2308013C031D19290319D9201D
:1001B00019291E08F039103A031DE028013086067F
:1001C0001E08F039203A031DE728023086061E0873
:1001D000F039303A031DEE28043086061E08F03947
:1001E000403A031DF528083086061E08F039503ABB
:1001F000031DFC28103086061E08F039603A031DE6
:100200000329203086061E08F039703A031D0A299A
:10021000403086061E08F039803A031D11298030CF
:1002200086061E08F039F03A031D1829803086062C
:10023000080026088A0025088300A40E240E080062
:10024000A4000308A5000A08A600A30126088A0046
:0A02500025088300A40E240E080008
:02400E00323D41
:00000001FF
